:0200000001B845
:0100030032CA
:02000B000134BE
:0100130032BA
:02001B0001766C
:0100230032AA
:01002B0032A2
:1000330032C000C0D0C0E0C083C0829002BFE56080
:100043002393F561A3E560230493F56285618C85B1
:10005300628AE560B41E097590FFD2B7C28C016B4A
:100063002440F8E6F5900560D082D083D0E0D0D06C
:10007300D00032C0D0C0E0D57B36757B28D57C302C
:10008300757C32200007D200754EEB8005C20075E7
:100093004EFFD57D1B757D78E574B43B0D757400FB
:1000A300E570B41709757000800605748002057049
:1000B300D0E0D0D032758107C2D3C2D5C2AF74FFAE
:1000C300787FF6D8FD758D06758B06758921758742
:1000D30080759850D28EC28CD288D28AD2ACD2A9E3
:1000E300D2ABD2AF7590FF75B0FF75700C7574000D
:1000F300756800756C00757B28757C32757D78207A
:100103000917EAB4010B120242856875856C788081
:100113000E75184012024C801F85707585747875B2
:100123001840120197E576512AE577512A7518523E
:10013300E579512AE57A512A79FF20B71ED9FB7553
:100143006000758CEB758A00D28C79FF30B7FBD9D0
:10015300FBC28C7590FF1201AE21027BFF7CFF3046
:10016300B7D8DCFBDBF7E56CB5741BE568B5701637
:10017300747F03F59012018E20E0F723F5901201AE
:100183008E20E6F721027590FF21027BFA7CFADCD0
:10019300FEDBFA22E57575F00A84F57685F077E5DE
:1001A3007875F00A84F57985F07A22E5B003034483
:1001B300F0B4FF11D9F52009031202427521FF752E
:1001C3005FFF7A0722D9E4B55F04DA5A7A01B4FEF5
:1001D30005F55FC20922B4FC0EF55FE568B41704A8
:1001E30075680022056822B4FA0EF55FE56CB43B2E
:1001F30004756C0022056C22B4F50EF55FE570B44E
:10020300170475700022057022B4F30EF55FE574D0
:10021300B43B0475740022057422B4F602F55FB48E
:10022300F704F55F7A072290027DA818790675F026
:1002330006A4C0E093F608A3D0E0D9F68818227884
:100243004074FFF608B85EFB2290025FA818791E7F
:10025300E4C0E093F608D0E004D9F62281EEEEEE96
:1002630081FFFFBE80BFFFFFDFABABAB87FF83F731
:10027300FBFBF7FF83FBE7FB87FFC1BEBEBEC1FFEE
:10028300FFBD80BFFFFFBD9EAEB6B9FFDDBEB6B6F4
:10029300C9FFE7EBED80EFFFD8BABABAC6FFC1B624
:1002A300B6B6CDFF9EEEF6FAFCFFC9B6B6B6C9FFE9
:1002B300D9B6B6B6C1FFFFFFFFFFFFFFFA3AFA4117
:1002C300FA4CFA5BFA6EFA84FA9FFABCFADDFB0089
:1002D300FB25FB4CFB75FB9EFBC8FB9EFB75FB4C98
:1002E300FB25FB00FADDFABCFA9FFA84FA6EFA5B8F
:1002F300FA4CFA41FA3AFA38F32CF3F4F64CF7785D
:10030300F8A4F96CFA34FA34FAFCFBC4FA34FA347C
:10031300FAFCFAFCFB60FAFCFBC4FA34F96CF8A4AF
:10032300F7DCF714F7DCF714F64CF584F4BCF3F4BC
:10033300F32CE6ACFA88FA9CFAB0FAC4FAD8FAECD1
:10034300FB00FB14FB28FB3CFB50FB64FB78FB8CA2
:10035300FB78FB64FB50FB3CFB28FB14FB00FAEC33
:10036300FAD8FAC4FAB0FA9CFA88FA74FA60FA4C2A
:00000001FF
